:1000000000308A00372900000A108A100A1182077E
:100010006B346F34623475347234613400340A10D6
:100020008A100A11820720342034203420343034DE
:10003000753473346534633400340A108A100A113D
:1000400082072034253434346C346434753473348A
:1000500065346334003421308400000803193D28DE
:100060000630F800F701F70B3328F80B32287B3005
:10007000F700F70B3928800B30288A117B282108DC
:1000800086008510051105140510A630F700F70B42
:10009000472800000034F03066000511851405146F
:1000A0000608F039AF00051005140608F039B00055
:1000B000051000306600300EF7000F30F7057708A6
:1000C0002F04F80000342108A200220886008510C1
:1000D000051105140510A20EF030A20522088600B5
:1000E000051405104B207808A200A21B72280034CA
:1000F0000530A1002B283030A1003F203030A10076
:100100003F203030A1003F202030A1003F202E3082
:10011000A10063200C30A10063200630A100632001
:100120008A114B292E088600851005150514051027
:10013000AE0EF030AE052E088600051405104B20DB
:100140007808AF00AF1B9F280034F801F901F701D0
:10015000FA012808031DAF2827080319C928103001
:10016000A9000310A50DA60DF70DFA0D28087A02B7
:10017000031DBC2827087702031CC5282708F7029F
:10018000031CFA032808FA020314F80DF90DA90B51
:10019000B12800008A11B3290408AD00A71FD9288F
:1001A0002D30AE0092208403A609A709A60A0319E0
:1001B000A70A270EF038A900A907E23EAA00323E9E
:1001C000AC0027080F39AA07AA07AC07E93EAB0025
:1001D000AB07AB07260E0F39AB07AC07AB0DAC0D69
:1001E000AC09AC0D26080F39AC07A90D0730A800E3
:1001F0000A30AC07AB03031CF928AB07AA03031CA6
:10020000FD28AA07A903031C0129A907A803031CA9
:1002100005292830840007302D0584072C3004027E
:1002200003192E290008F700031D1C292D1A2C295B
:10023000AD191E2920301F290830AD003030F707D6
:10024000A7010408A6007708A8007708AE0092204E
:10025000260884002808F700840A0E290008F70001
:100260003030F7077708AE0092208A11C129840147
:100270001F30830507309F008316050883121F086F
:100280000C13953090001010383065000030660077
:10029000850186017828A10121080F200038031963
:1002A0005529A10AAE0092204C29CA30A100632032
:1002B000A10121080420003803196229A10AAE0017
:1002C000922059298F018E01851D64291014851DE6
:1002D0006E290F081D3C031C6E29672910100F089A
:1002E0001C3C03186229A001051E2014851EA014C1
:1002F0008F018E012008FC3E0318CF29043ED1292E
:1003000085198029851D822985198429851D8629BD
:1003100085198829851D8A2985198C291014851D20
:100320008F298519912910108030A10063200F08B2
:10033000FA000E08F7000F087A02031D97297708C4
:10034000A1007A08A200210DA300220DA400A30D94
:10035000A40DFC30A3052408A6002308A500A801CD
:100360000A30A700A5287908A5007808A400203045
:10037000AE009220013084002508A7002408A600C2
:10038000CC280530A60026081D20A60AF70077080D
:10039000AE00922009302602031DC329CF2962290D
:1003A00063000A148A100A1182078C29882984297B
:0203B0008029A2
:02400E00423F2F
:00000001FF
